:100000000C942B000C9453000C9453000C9453004C
:100010000C9453000C9453000C9453000C94530014
:100020000C9453000C9453000C9453000C94530004
:100030000C9453000C9453000C9453000C945300F4
:100040000C9453000C9453000C9453000C945300E4
:100050000C945300F20011241FBECFE5D4E0DEBFA4
:10006000CDBF10E0A0E6B0E0E6E3F8E002C0059006
:100070000D92A637B107D9F720E0A6E7B0E001C09E
:100080001D92A637B207E1F710E0C6E5D0E004C044
:100090002297FE010E944001C435D107C9F70E9492
:1000A000A0000C9419040C940000FC0103C05D9B9B
:1000B000FECF8CB981918111FACF0895A39A08954A
:1000C000AB9A0895282F98E080E027FF02C0A99AF4
:1000D00001C0A998A19A880F9C998160AA9AA29AB6
:1000E000220F00C00000AA98A29A915071F70895BB
:1000F000EF92FF921F93CF93DF9300D0CDB7DEB77F
:10010000182FAB989A830E945E008A810E94620039
:10011000F82EE12C812F0E9462009701282BC90143
:100120008A8399830E9460000E945E008A8199817F
:100130000F900F90DF91CF911F91FF90EF90089556
:10014000CF93DF93CDB7DEB72A970FB6F894DEBF13
:100150000FBECDBF88EC92E80E94780081E89AEC4F
:100160000E94780083E89AEC0E94780080E6E82EEE
:1001700080E0F82E8E010F5F1F4F18C0A89A2FEF56
:1001800080E792E0215080409040E1F700C00000FD
:10019000A8982FEF80E792E0215080409040E1F74F
:1001A00000C0000085E690E00E945500AB980E94D8
:1001B0005E009C9BE3CF80E090EB0E947800992743
:1001C0009F938F93FF92EF921F930F930E9444018E
:1001D000C8010E9455000F900F900F900F900F9044
:1001E0000F90E4CFA09AA898789483E389B988E027
:1001F0008AB986E880BD88E690E00E945500A998FB
:10020000A19AAA98A29A0E9460000E945E00A498F7
:10021000AC982FEF80E792E0215080409040E1F7CA
:1002200000C0000080EE90EC0E94780087ED90E81E
:100230000E9478008BEA92EC0E94780081E89AECA8
:100240000E94780080E090EE0E94780080E098ECB8
:100250000E94780087EF94EC0E94780080E296EA92
:100260000E94780087E294E90E94780082E296EC8E
:100270000E94780080E698E90C947800EE0FFF1F4A
:100280000590F491E02D0994AEE0B0E0EAE4F1E0ED
:100290000C94F0030D891E8986E08C831A830983F0
:1002A0008FEF9FE79E838D83CE014996AC016F89C6
:1002B000788DCE0101960E946601EF81F885E00FEE
:1002C000F11F10822E96E4E00C940C04ACE0B0E038
:1002D000ECE6F1E00C94E2037C016B018A01FC0185
:1002E00017821682838181FFC6C188248394912C52
:1002F0008C0E9D1EF7019381F60193FD859193FF6E
:1003000081916F01882309F4B2C1853239F493FDDC
:10031000859193FF81916F01853229F4B70190E0B7
:100320000E945803E7CF512C312C20E02032A8F452
:100330008B3261F028F4803251F0833271F40BC0BB
:100340008D3239F0803349F4216028C02260246066
:1003500025C0286023C0206121C027FD27C0382F79
:1003600030533A3078F426FF06C0FAE05F9E300D35
:100370001124532E13C08AE0389E300D1124332EE1
:1003800020620CC08E3221F426FD71C1206406C0AB
:100390008C3611F4206802C0883641F4F60193FDD2
:1003A000859193FF81916F018111C0CF982F955452
:1003B000933018F09052933028F40C5F1F4FFFE3F6
:1003C000F9830DC0833631F0833771F0833509F03E
:1003D0005EC023C0F801808189830E5F1F4F4424D3
:1003E0004394512C540115C03801F2E06F0E711C7A
:1003F000F801A080B18026FF03C0652D70E002C027
:100400006FEF7FEFC5012C870E944D032C01830104
:100410002C856FE7262E222218C03801F2E06F0EDD
:10042000711CF801A080B18026FF03C0652D70E02B
:1004300002C06FEF7FEFC5012C870E9442032C01A1
:100440002C8550E8252E222A830123FC1CC006C0DF
:10045000B70180E290E00E9458033A94832D90E027
:1004600048165906A8F30FC0F50127FC859127FE11
:1004700081915F01B70190E00E94580331103A94D6
:10048000F1E04F1A51084114510471F7EDC0843660
:1004900011F0893641F5F80127FF07C060817181AD
:1004A000828193810C5F1F4F08C060817181882712
:1004B00077FD8095982F0E5F1F4F4FE6B42EB22226
:1004C00097FF09C090958095709561957F4F8F4FEC
:1004D0009F4FF0E8BF2A2AE030E0A4010E94840385
:1004E000A82EA81843C0853731F43FEEB32EB222B0
:1004F0002AE030E024C099EFB92EB2228F36B9F04D
:1005000020F4883509F0B3C00DC0803721F088375A
:1005100009F0ADC002C020E1B22AB4FE0BC084E0F5
:10052000B82A08C024FF09C0E6E0BE2A06C028E0B9
:1005300030E005C020E130E002C020E132E0F80107
:10054000B7FE07C060817181828193810C5F1F4F6C
:1005500006C06081718180E090E00E5F1F4FA401B2
:100560000E948403A82EA818FFE7BF22B6FE0BC086
:100570002B2D2E7FA51450F4B4FE0AC0B2FC08C087
:100580002B2D2E7E05C07A2C2B2D03C07A2C01C07A
:10059000752C24FF0DC0FE01EA0DF11D8081803312
:1005A00011F4297E09C022FF06C07394739404C01D
:1005B000822F867809F0739423FD14C020FF0FC0AA
:1005C0005A2C731460F4530C5718732C08C0B701DD
:1005D00080E290E02C870E94580373942C8573145A
:1005E000B0F304C0731410F4371801C0312C24FF89
:1005F00012C0B70180E390E02C870E9458032C853D
:1006000022FF1EC021FF03C088E590E002C088E7FA
:1006100090E0B7010CC0822F867891F021FD02C0D6
:1006200080E201C08BE227FD8DE2B70190E00E94DD
:10063000580306C0B70180E390E00E9458035A9423
:10064000A514C0F3AA94F401EA0DF11DB70180814D
:1006500090E00E945803A110F5CF06C0B70180E2D8
:1006600090E00E9458033A943110F8CF43CEF7013E
:100670002681378102C02FEF3FEFC9012C96E2E1BE
:100680000C94FE03FC010590615070400110D8F7F6
:10069000809590958E0F9F1F0895FC0161507040CA
:1006A00001900110D8F7809590958E0F9F1F0895A7
:1006B0000F931F93CF93DF938C01EB018B8181FD0F
:1006C00003C00FEF1FEF1AC082FF0DC02E813F81C4
:1006D0008C819D812817390764F4E881F9810193A1
:1006E000F983E88306C0E885F985802F0995892B71
:1006F00041F78E819F8101969F838E83C801DF9190
:10070000CF911F910F910895FA01AA27283051F136
:10071000203181F1E8946F936E7F6E5F7F4F8F4F32
:100720009F4FAF4FB1E03ED0B4E03CD0670F781F91
:10073000891F9A1FA11D680F791F8A1F911DA11D76
:100740006A0F711D811D911DA11D20D009F46894AF
:100750003F912AE0269F11243019305D3193DEF657
:10076000CF010895462F4770405D4193B3E00FD00D
:10077000C9F7F6CF462F4F70405D4A3318F0495DF8
:1007800031FD4052419302D0A9F7EACFB4E0A695DB
:100790009795879577956795BA95C9F700976105FD
:1007A000710508959B01AC010A2E06945795479553
:1007B00037952795BA95C9F7620F731F841F951F48
:1007C000A01D08952F923F924F925F926F927F9259
:1007D0008F929F92AF92BF92CF92DF92EF92FF9251
:1007E0000F931F93CF93DF93CDB7DEB7CA1BDB0BFD
:1007F0000FB6F894DEBF0FBECDBF09942A883988A2
:1008000048885F846E847D848C849B84AA84B984A8
:10081000C884DF80EE80FD800C811B81AA81B981B4
:10082000CE0FD11D0FB6F894DEBF0FBECDBFED01C8
:060830000895F894FFCFCB
:1008360025303458200D0A005561727420646F6E9D
:0608460065210D0A00000F
:00000001FF
